:1000000002095F7DA37C08ED1D70011C144C70F784
:10001000EF1F70011E144E70EA224101C700C10992
:0100200000DF
:10002300020A559001CA7401F074FFA3F0A3F0A370
:100033007401F0A37407F0A37409F07B017A0179CA
:10004300CA120B45E4FBFD7F01120B8F43BA80906C
:10005300FA11E04440F053BA7F22EF640170044385
:07006300BC802253BC7F2288
:10006B00020BD6120106120C2B120C02120026D216
:10007B00AF7FC87E001200033009F6C209E490017D
:10008B00C8F09001C8E0C39410748094805053E47E
:10009B00A3F09001C9E0FFC3940C7480948050319D
:1000AB007BFF7A0C79539001C8E075F00CA4240700
:1000BB00F582E43401F583E5822FF582E43583F58F
:1000CB0083E09001CDF012024A9001C9E004F08068
:1000DB00C17BFF7A0C795C12024A9001C8E004F0F4
:1000EB0080A07BFF7A0C795C12024A43BA8090FAAB
:1000FB0011E04440F053BA7F02007C43937F53944A
:10010B00807591FF75920053B1FC53B2FC228F990D
:0D011B009000037401F0900003E070FA22E0
:07012B0021DDAE07020119FE
:0201330021DDCC
:02013B0021DDC4
:0201430021DDBC
:02014B0021DDB4
:0201530021DDAC
:02015B0021DDA4
:020163008078A2
:02016B008070A2
:020173008068A2
:02017B008060A2
:020183008058A2
:02018B008050A2
:020193008048A2
:02019B008040A2
:0201A3008038A2
:0201AB008030A2
:0201B3008028A2
:0201BB008020A2
:0201C3008018A2
:0201CB008010A2
:0201D3008008A2
:1001DB008000016BE50824CDF582E43401F583E062
:1001EB000508229001CA3007039001CDE475F00198
:1001FB001207690205442000E97F2ED2008018EF18
:10020B00540F2490D43440D4FF30040BEF24BFB4EC
:10021B001A0050032461FFE50960021509050CE57E
:10022B000C7002050B30070E9001CAE475F0011239
:10023B000769EF02072102012D7403D2078003E443
:10024B00C207F5089001CA120780E4F509F50BF512
:10025B000CE50960077F2012022280F5750AFFC2A8
:10026B0001C200C202C203C205C206C2081201EEDD
:10027B00FF700D3007057F00120233AF0CAE0B225F
:10028B00B4255FC2D5C2041201EEFF24D0B40A001C
:10029B00501A75F00A780930D50508B6FF0106C665
:1002AB00A426F620D5047002D20380D924CFB41A29
:1002BB0000EF5004C2E5D204020434D20180C6D24E
:1002CB000080C0D20280BCD2D580BAD20580B47F68
:1002DB00201202222002077401B5090040F112011D
:1002EB00DFFF12022202025CD208D20680951201B5
:1002FB00DFFB1201DFFA1201DFF94A4B70067905B9
:10030B007A057BFF20022EE509602A7E008E82751E
:10031B00830012055D60060EEE650A70F0C2D5EB28
:10032B00C0E0EAC0E0E9C0E0EE12047BD0E0F9D017
:10033B00E0FAD0E0FB120544FF60AAEBC0E0EAC094
:10034B00E0E9C0E0120222D0E02401F9D0E0340051
:10035B00FAD0E0FBE50A0460DCD50AD980877BFF85
:10036B007A047977D202809C791080027908C206D0
:10037B00C2088008D2D5790A8004790AC2D5E50A69
:10038B00047002F50AE4FAFDFEFF1201DFFC7B08A4
:10039B002001131201DFFD7B1030000A1201DFFE7A
:1003AB001201DFFF7B20EC3382D592D55013C3E4CF
:1003BB003000069FFFE49EFEE42001039DFDE49CBC
:1003CB00FCE4CBF8C201EC700CCFCECDCCE824F81A
:1003DB00F870F38017C3EF33FFEE33FEED33FDEC14
:1003EB0033FCEB33FB994002FB0FD8E9EB300105F3
:1003FB00F8D0E0C448B201C0E00AEC4D4E4F782073
:10040B007B0070C2EAB50A0040BCC0E012047DD08C
:10041B00F0D0E0200104C4C0E0C4B201C0F012026D
:10042B000BD0F0D5F0EB02025C12078902F95303F3
:10043B00735802CA4C02C64203774F037F44037FB3
:10044B004902DF4303855503694603694503694741
:10045B0005255002CE2D02D22E02F52B02D62302F9
:10046B00F320050E2A028E48000002ED3F3F3F00AD
:10047B00790AA2D5200314300509B910020404B976
:10048B00080104A2D5200602500104200268920242
:10049B00B509005034C0E07F203003197F30A20231
:1004AB0072067205500F1204D4C202C206C205C2F4
:1004BB00087F30800F300503E9C0E01202223005BF
:1004CB0003D0E0F9D0E0B509CC3005177F30B91077
:1004DB000C1202227F583004077F788003B908037F
:1004EB001202223002057F2D0202227F202008F803
:1004FB007F2B2006F322920280CF286E756C6C291D
:10050B0000D2011201DF3001F8C201780930D501A8
:10051B0008F602028E2D504349581201DF2403B412
:10052B0005004001E490052093120213743A120265
:10053B0013D203750904020373BB010689828A83F4
:10054B00E0225002E722BBFE02E32289828A83E487
:10055B009322BB010CE58229F582E5833AF583E012
:10056B00225006E92582F8E622BBFE06E92582F831
:10057B00E222E58229F582E5833AF583E49322BBF7
:10058B000110E58229F582E5833AF583E0F5F0A3C6
:10059B00E0225009E92582F886F008E622BBFE0A24
:1005AB00E92582F8E2F5F008E222E5832AF583E9F2
:1005BB0093F5F0A3E9932275F008758200EF2FFFF6
:1005CB00EE33FECD33CDCC33CCC58233C5829BED20
:1005DB009AEC99E58298400CF582EE9BFEED9AFD24
:1005EB00EC99FC0FD5F0D6E4CEFBE4CDFAE4CCF9D4
:1005FB00A88222B800C1B90059BA002DEC8BF08447
:10060B00CFCECDFCE5F0CBF97818EF2FFFEE33FE14
:10061B00ED33FDEC33FCEB33FB10D703994004EBCC
:10062B0099FB0FD8E5E4F9FA227818EF2FFFEE3398
:10063B00FEED33FDEC33FCC933C910D7059BE99AAA
:10064B004007EC9BFCE99AF90FD8E0E4C9FAE4CC3B
:10065B00FB2275F010EF2FFFEE33FEED33FDCC33A5
:10066B00CCC833C810D7079BEC9AE899400AED9B8E
:10067B00FDEC9AFCE899F80FD5F0DAE4CDFBE4CC6D
:10068B00FAE4C8F922EB9FF5F0EA9E42F0E99D42AD
:10069B00F0E89C45F022E8600FECC313FCED13FD72
:1006AB00EE13FEEF13FFD8F122BB010DE58229F506
:1006BB0082E5833AF5830207405007E92582F80269
:1006CB000733BBFE07E92582F802074CE58229F5C3
:1006DB0082E5833AF583020759ECF0A3EDF0A3EE24
:1006EB00F0A3EFF022A8828583F0D083D08212078B
:1006FB0007120707120707120707E473E493A3C552
:10070B0083C5F0C583C8C582C8F0A3C583C5F0C532
:10071B0083C8C582C822BB010689828A83F0225016
:10072B0002F722BBFE01F322E6FB08E6F908E6FA24
:10073B0008E6CBF822E0F8A3E0F9A3E0FAA3E0FB8C
:10074B0022E2FB08E2F908E2FA08E2CBF822E49392
:10075B00F8740193F9740293FA740393FB22F8E093
:10076B00FBA3A3E0F925F0F0E58215827002158357
:10077B00E0FA38F022EBF0A3EAF0A3E9F022D08301
:10078B00D082F8E4937012740193700DA3A393F8C5
:10079B00740193F5828883E4737402936860EFA30A
:1007AB00A3A380DF9001D3EBF0A3EAF0A3E9F0EF72
:1007BB006401600302095C90000004F0E4A3F0A361
:1007CB00F0A3F0A3F0A3F0A3F0FFEFC39480748029
:1007DB009480500F74872FF582E43400F583E4F096
:1007EB000F80E7E4FFEFC3948074809480500F7404
:1007FB00072FF582E43400F583E4F00F80E79001D6
:10080B00D3E0FBA3E0FAA3E0F9120544FFE598540B
:10081B003F4FF598EF64C06008EF64406003020936
:10082B00019000021206B47F007E607D547C0012A2
:10083B0005FE9001D61206E4E4FFFE7D01FC90015B
:10084B00D6E0F8A3E0F9A3E0FAA3E0FBC31206900D
:10085B0040037FFF229001D6E0F8A3E0F9A3E0FA72
:10086B00A3E0FBC3E49BFFE49AFE740199FDE498BB
:10087B00FC9001D61206E49001D3E0FBA3E0FAA3AF
:10088B00E0F990000112055D64027032538EEF4364
:10089B008E01538EF7438E049001D6E0FCA3E0FD4E
:1008AB00A3E0FEA3E0FF78081206A18FD69001D635
:1008BB00A3A3A3E0F5D753AFFB438E108077C28E73
:1008CB00538EFE5389BF5389CF438E409001D6E0A0
:1008DB00FCA3E0FDA3E0FEA3E0FF78081206A18FC6
:1008EB008D9001D6A3A3A3E0F58BC2AB5389BF5365
:1008FB008FFDD28E803F9001D3E0FBA3E0FAA3E003
:10090B00F9120544FF7E00701490000812055D6417
:10091B00017005438E20801D538EDF8018EF64809D
:10092B004E701290000812055D64017005438780BC
:10093B00800353877F9001D3E0FBA3E0FAA3E0F998
:10094B0090000712055D7004C29C8002D29C7F0050
:10095B00227FFF22787FE4F6D8FD7581210209A65C
:10096B0002006EE493A3F8E493A34003F68001F234
:10097B0008DFF48029E493A3F85407240CC8C3338D
:10098B00C4540F4420C8834004F456800146F6DF5C
:10099B00E4800B010204081020408090001AE47ED2
:1009AB00019360BCA3FF543F30E509541FFEE49351
:1009BB00A360010ECF54C025E060A840B8E493A318
:1009CB00FAE493A3F8E493A3C8C582C8CAC583CA43
:1009DB00F0A3C8C582C8CAC583CADFE9DEE780BEFB
:1009EB0090000112055DFFE5DE54F04FF5DE90003F
:1009FB000212055DC43354E0FFE5DE54DF4FF5DE34
:100A0B00120544D3941F74809480503D90000312C0
:100A1B00055DFFD3940174809480502D90000412D7
:100A2B00055DFED3940374809480501D43BA80EE11
:100A3B00C43354E0FEEFC433333354804EFF1205FE
:100A4B00444F90FEA8F053BA7F22C0E0C083C0820F
:100A5B00C0D075D000C007309831C298900006E026
:100A6B007029900004E0C39480748094804002E469
:100A7B00F0900004E0FF04F074072FF582E43400DB
:100A8B00F583E599F09000057405F0309907C2994C
:100A9B00900003E4F0D007D0D0D082D083D0E032E6
:100AAB00EFFBD39401748094805009EB7004C2ADBA
:100ABB008002D2ADEDFF7E00D394037480948050FE
:100ACB0029EF700553B7DFC2BDEF64014E700553BC
:100ADB00B7DFD2BDEF64024E700543B720C2BDEF46
:100AEB0064034E700543B720D2BD7F0022EFFBD3CA
:100AFB009401748094805009EB7004C2AC8002D2D4
:100B0B00ACEDFF7E00D39403748094805029EF707A
:100B1B000553B7EFC2BCEF64014E700553B7EFD26C
:100B2B00BCEF64024E700543B710C2BCEF64034EBA
:100B3B00700543B710D2BC7F002243BA8090FA12E3
:100B4B00E4F090000112058AFF90FA1AE5F0F0A389
:100B5B00EFF090000312058AFF90FA17E5F0F0A36F
:100B6B00EFF090000512055D90FA19F01205446440
:100B7B000190FA117006E04480F08004E0547FF09D
:100B8B0053BA7F2243BA8090FA10E054F0F0EDD3C1
:100B9B00940374809480500BE0FEED25E025E0FD7E
:100BAB00EE4DF0EBD3940374809480500690FA10C2
:100BBB00E04BF0EF640190FA107006E04480F08097
:100BCB0004E0547FF053BA7F7F0022C0E0C083C0A3
:100BDB0082C0D075D000C007AFBA43BA8090FA126A
:100BEB00E030E006E054FEF0D2098FBAD007D0D047
:100BFB00D082D083D0E0329001CA741FF0E4900110
:100C0B00CDF0A304F0E49001CBF0A304F0FB7A0148
:100C1B0079CA1209EB7F0112005DE4FDFF020AABFA
:100C2B009001CA7440F0A37401F0A31206F0000106
:100C3B00C2009001D17401F0FB7A0179CAFF12074F
:100C4B00AF7D017F01020AF83078253032627820BF
:040C5B00000D0A007E
:00000001FF
